:10000000F6EF04F00000000000EF00F00000000038
:0A0010000000000000000000F3D71C
:0C001C0072B201D0FDD725C173FF1200A5
:1000280001012551030A00E12551040A00E1255187
:0C003800050A00E12551060A00E1120053
:0E004400ACB202D00000FCD725C1ADFF120007
:10005200C7B409D01F0EC514016E0150000A03E196
:0A006200010E006E01D0006A1200CA
:10006C00F250026EF29E0500FF6A0150FE6E0050C7
:08007C00FD6E02BEF28E1200BF
:1000840039C021F13AC022F13BC023F13CC024F134
:1000940001011F6B206B2051120802E11F518E08D1
:1000A40008E3D5DF005201E004D001011F4B202BEF
:1000B400F2D70101120E205D02E18F0E1F5D03E3F2
:1000C4007B0E006E24D0C580C5A020D039503A10D4
:1000D4003B103C101AE021512211231124110EE18E
:1000E400F4C0E1FFF5C0E2FF050EE66EF2C000F0D9
:1000F400F3C001F0B9DF010E006E09D0010E010159
:10010400215F000E225B235B245BDED7006A1200B2
:04011400C58412008C
:100118009E961FC1C9FF39C020F13AC021F13BC0EA
:1001280022F13CC023F1C7A421D039503A103B102A
:100138003C101BE0010120512111221123110EE175
:10014800F4C0E1FFF5C0E2FF040EE66EF2C000F075
:10015800F3C001F087DF010E006E3AD0010E0101F5
:10016800205F000E215B225B235BDDD739C020F1C5
:100178003AC021F13BC022F13CC023F19EB621D008
:1001880039503A103B103C101BE00101205121115D
:10019800221123110EE1F4C0E1FFF5C0E2FF040EC5
:1001A800E66EF2C000F0F3C001F05CDF010E006EF5
:1001B8000FD0010E0101205F000E215B225B235B43
:1001C800DDD7C5BC02D0006A03D0C584020E006E1C
:0201D800120013
:1001DA00086A080E0C6E003408360450085ED8B05F
:0E01EA0002D00826D89000360C2EF5D7120051
:1001F80001011E6BF00E1B151C6F1BC11DF11D3775
:100208001D911D371D911D371D911D371D91F00E34
:100218001D1734DF1ADF4E0E01011F6F79DF15DF5E
:1002280001011E511C111F6F1F851F8771DF0DDF14
:10023800420E0D6E0D2EFED7000001011E511C113D
:100248001F6F1F8765DF01DF850E0D6E0D2EFED730
:1002580001011E511D111F6F1F851F8759DFF5DE14
:10026800420E0D6E0D2EFED7000001011E511D110C
:100278001F6F1F874DDFE9DE49DF01011B51010AAE
:1002880009E10B0E0C6E620E0D6E0D2EFED70C2EB4
:06029800FCD7000012007B
:10029E0015C100F00032009E0032009E0032009E1A
:1002AE000032009E2B0E0024F66E100EF76E000E1E
:1002BE00F722000EF86E000EF8220900F5CF00F0BE
:1002CE0016C1E1FF17C1E2FF00C0E6FF010E0101FA
:1002DE001625E16E000E1721E26E0F0E1515006E3B
:1002EE002B0E0024F66E100EF76E000EF722000E87
:1002FE00F86E000EF8220900F5CF00F000C0E6FF00
:10030E00020E1625E16E000E1721E26EE66A12004D
:10031E0015C1F6FF16C1F7FF17C1F8FF0900F5CF9B
:10032E0018F101011851000818E215C1F6FF16C1A7
:10033E00F7FF17C1F8FF0900F5CF00F000C018F164
:10034E00010E1527000E1623172300C025F173DEAC
:0C035E00850E0D6E0D2EFED7E4D71200A8
:10036A00010E01011A6F1CD01605006E0050800F95
:10037A001B6F3DDF21D01605006E0050C00F1B6FAA
:10038A0036DF1AD01605006E0050940F1B6F2FDF50
:10039A0013D01605006E0050D40F1B6F28DF0CD047
:1003AA001551010AE1E01551020AE5E01551030A67
:1003BA00E9E01551040AEDE0F00E1715186F17C1A0
:1003CA0019F11937199119371991193719911937DB
:1003DA001991F00E191751DE37DE4E0E01011F6F0B
:1003EA0096DE32DE01011A5118111F6F1F851F8711
:1003FA008EDE2ADE420E0D6E0D2EFED700000101A2
:10040A001A5118111F6F1F8782DE1EDE850E0D6EB0
:10041A000D2EFED701011A5119111F6F1F851F8753
:10042A0076DE12DE420E0D6E0D2EFED700000101A1
:10043A001A5119111F6F1F876ADE06DE66DE120067
:10044A000D0E0101256FF9DD0A0E0101256FF5DD9B
:02045A0012008E
:10045C0015C102F016C103F002C000F003C001F098
:10046C00024A032A00C0E9FF01C0EAFFEE5201E094
:10047C00F3D701011551025C006E16510358016E41
:0A048C00010E005E000E015A12007E
:1004960017C1F6FF18C1F7FF19C1F8FF0900F5CF1C
:1004A60000F0005218E017C1F6FF18C1F7FF19C196
:1004B600F8FF0900F5CF00F015C1E1FF16C1E2FF14
:1004C60000C0E6FF0101154B162B010E1727000E83
:1004D60018231923DDD715C1E1FF16C1E2FFE66A2D
:0204E600120002
:1004E80015C104F016C105F004C0E9FF05C0EAFF14
:1004F800EE5203E0044A052AF7D704C002F005C00B
:1005080003F0044A052A17C100F018C101F00101DF
:10051800174B182B00C0E9FF01C0EAFF02C0E1FF3A
:1005280003C0E2FFEECFE6FF02C0E9FF03C0EAFF27
:10053800EE5201E0E2D715C100F016C101F0120039
:100548000101186B030E185D0AE218511625E16EB9
:10055800000E1721E26E200EE66E182BF3D7185105
:100568001625E16E000E1721E26EE66A180718518B
:100578001625196F000E17211A6F0A0E046E15C181
:1005880000F027DE08C000F0300E002619C1E1FF98
:100598001AC1E2FF00C0E6FF0A0E046E15C100F0A2
:1005A80018DE00C015F10050000A01E102D018075A
:0405B800DED7120078
:1005BC000101186B15C1E9FF16C1EAFFEECF17F167
:1005CC001751000A0EE017C125F136DD0101182B79
:1005DC0018511525E96E000E1621EA6EEECF17F1B3
:0405EC00EFD7120033
:1005F000440E0101016F000E026F250E036F010E04
:10060000046FFF0E0001F96FFF0EFA6F000EFB6F13
:10061000000EFC6FFF0E0101096FFF0E0A6F000E46
:100620000B6F000E0C6FFF0E056FFF0E066F000EB6
:10063000076F000E086FAC8A900EAB6E948E949C80
:0C0640009EAA03D0AECF00F0FBD7120042
:10064C00520E0001EE6F000EEF6F000EF06F000EF9
:10065C00F16F840EEA6F000EEB6F000EEC6F000E64
:10066C00ED6FFF0EE66FFF0EE76F000EE86F000EEA
:10067C00E96FFF0EE06FFF0EE16FFF0EE26FFF0EF2
:10068C00E36F180ED86F010ED96F1F0EDA6F010EC3
:10069C00DB6F140EDC6F010EDD6F000EDE6F000ED3
:1006AC00DF6F949894968B988B9694889486C79EBB
:0806BC00C79C380EC66E120047
:1006C4000900F5CFE6FF0006FBE10106F9E112009F
:1006D400806A0F01386B38813883E30E926E396B70
:1006E400FF0E816EFF0E936E796A786A826A3A6BA6
:0C06F400800E946E956A3B6B606A1200E9
:100700000FC1E9FF10C1EAFFEE5210E00DC115F173
:100710000EC116F10FC1E9FF10C1EAFFEECF17F1CC
:0E07200024DE01010E2B0F4B102BEAD7120026
:10072E000001FD6BA8DC8EDC4E0E01011F6FEDDCAF
:10073E0089DC9C0E0C6ED70E0D6E0D2EFED70C2E78
:10074E00FCD7300E0001FD1101011F6F1F851F87A1
:10075E00DCDC78DC420E0D6E0D2EFED70000300E66
:10076E000001FD1101011F6F1F87CFDC6BDC340E02
:10077E000C6EF10E0D6E0D2EFED70C2EFCD700005A
:10078E000000300E0001FD1101011F6F1F851F8734
:10079E00BCDC58DC420E0D6E0D2EFED70000300E66
:1007AE000001FD1101011F6F1F87AFDC4BDC340E02
:1007BE000C6EF10E0D6E0D2EFED70C2EFCD700001A
:1007CE000000300E0001FD1101011F6F1F851F87F4
:1007DE009CDC38DC420E0D6E0D2EFED70000300E66
:1007EE000001FD1101011F6F1F878FDC2BDC340E02
:1007FE000C6EF10E0D6E0D2EFED70C2EFCD70000DA
:10080E000000200E0001FD1101011F6F1F851F87C3
:10081E007CDC18DC420E0D6E0D2EFED70000200E75
:10082E000001FD1101011F6F1F876FDC0BDC6BDCFC
:10083E00340E0C6EF10E0D6E0D2EFED70C2EFCD757
:10084E0000000000280E01011B6FCFDC060E1B6F8F
:04085E00CCDC1200DC
:100862000DC139F00EC13AF00FC13BF010C13CF09E
:1008720011C1F2F012C1F3F013C1F4F014C1F5F09A
:02088200120062
:100884000101006B0001FE51000826E2D4C015F1FD
:10089400D5C016F1610E0101176F100E186F000E0E
:1008A400196FF7DDD4C015F1D5C016F1D5DDFDC043
:1008B40015F1AB0E166F000E176F44DED4C015F1A0
:1008C400D5C016F1AB0E176F000E186F0BDED4C037
:1008D40015F1D5C016F170DEC69E42EC00F0FDC0E5
:1008E4001FF118DC00C0FFF0000E016EFF0E0118AE
:1008F40002E1FF0E001803E1C9CFFFF0C69E08DC39
:100904000001FF51000A0FE00101006B0001FE51DC
:10091400000808E2560E0101156F100E166F000E46
:10092400176FFBDC44D0010E0101006FCB0E0001F8
:10093400D625E16E000ED721E26EFDC0E6FFFE5122
:10094400000832E2AB0E0101156F000E166FBA0EED
:10095400176F0F0E186F000E196F9BDD300E00011C
:10096400D625B46FFDC015F1C00E0101166F000E3F
:10097400176FE8DDAB0E156F000E166F1DDE6B0EE4
:10098400156F100E166F000E176FC7DCFDC015F142
:10099400AB0E0101166F000E176F7FDCAB0E156FE7
:1009A400000E166F09DE4FDD0001D64BD72B8AEC03
:1009B40000F0020E0B6E040E0C6EBA0E0D6E0D2EB0
:1009C400FED70C2EFCD70B2EFAD7000029EC00F032
:1009D4000050000A01E1FAD70001FE51000801E2CB
:0809E40032DD00C100F0120039
:1009EC0039EC08F0D36AD38CD38AD388D382D390D2
:1009FC009B6A9B9C150E0B6E4B0E0C6EBE0E0D6EF9
:100A0C000D2EFED70C2EFCD70B2EFAD70000F29E23
:100A1C005BDE150E0B6E4B0E0C6EBE0E0D6E0D2EA0
:100A2C00FED70C2EFCD70B2EFAD700000001E46B7E
:100A3C00E56B000EE55D02E1200EE45D0AE2AB0E13
:100A4C00E425E16E000EE521E26EE66AE44BE52B4F
:100A5C00F0D7E46BE56B000EE55D02E1500EE45D52
:100A6C000AE25B0EE425E16E000EE521E26EE66A19
:100A7C00E44BE52BF0D7E46BE56B000EE55D02E192
:100A8C00080EE45D0AE2CB0EE425E16E000EE521D2
:100A9C00E26EE66AE44BE52BF0D7E46BE56BD66BC4
:100AAC00D76B5B0ED46F000ED56FB886B06ACF0EC5
:100ABC00AF6EAC8497DD0C0E256F22EC00F00B0EA4
:100ACC000B6E260E0C6E5D0E0D6E0D2EFED70C2EC3
:100ADC00FCD70B2EFAD700000000B1DC190E010177
:100AEC00156F100E166F000E176F13DCA8DC940E2A
:100AFC000101156F0D0E166F000E176F0ADCF20E4A
:100B0C000101156F0F0E166F000E176F02DC690EC8
:100B1C000101156F0E0E166F000E176F8FEC01F0A2
:100B2C005D0E0101156F0F0E166F000E176F8FEC17
:100B3C0001F0EA0E0101156F0E0E166F000E176F05
:100B4C008FEC01F07CDC270E0101156F0E0E166F79
:100B5C00000E176F8FEC01F04B0E0101156F100E8C
:100B6C00166F000E176F8FEC01F0AA0E0101156FB6
:100B7C000E0E166F000E176F8FEC01F0D80E0101E0
:100B8C00156F0F0E166F000E176F8FEC01F0920E93
:100B9C000101156F0F0E166F000E176F8FEC01F021
:100BAC004EDC280EC86E4CDDB80E01010D6F0B0E1D
:100BBC000E6F000E0F6F106F280E116F000E126F5C
:100BCC00250E136F010E146F46DE8AEC00F0000147
:100BDC00E46BE56B010EF66F000EF76FD66BD76BFF
:100BEC00060E0101156F100E166F000E176F8FECAD
:100BFC0001F0000E80BA010E0101256F300E252781
:100C0C0022EC00F01CDC200E3D6EFE0E3D5C22E260
:100C1C0080BA09D03DC0FDF0010E0001FE6F2CDE44
:100C2C0000C0F8F007D03DC0FDF00001FE6B24DEE3
:100C3C0000C0F8F0020E0B6E040E0C6EBA0E0D6EA8
:100C4C000D2EFED70C2EFCD70B2EFAD70000020E61
:100C5C003D26DBD725EC02F0260E0101156F0F0E99
:100C6C00166F000E176F8FEC01F00001D66BD76B6F
:100C7C00000ED75D02E1080ED65D38E2AB0E010125
:100C8C00156F000E166F3B0E176F100E186F000EBF
:100C9C00196F4BEC02F0310E0001D625B46FCB0E60
:100CAC00D625E96E000ED721EA6EEE50000810E250
:100CBC00CB0ED625E96E000ED721EA6EEECF15F1DC
:100CCC00B80E0101166F000E176F4FEC01F002D039
:100CDC000001B66BAB0E0101156F000E166F68DCD0
:100CEC0025EC02F00001D64BD72BC2D725EC02F035
:100CFC00150E0B6E4B0E0C6EBE0E0D6E0D2EFED722
:100D0C000C2EFCD70B2EFAD700000BDD0C0E1B6F34
:100D1C00FCEC00F0010E1B6FFCEC00F0150E0B6EE2
:100D2C004B0E0C6EBE0E0D6E0D2EFED70C2EFCD780
:100D3C000B2EFAD70000010E0D6F010E0E6F4D0E2B
:100D4C000F6F000E106FD6DC020E01010D6F010E3D
:100D5C000E6F3E0E0F6F000E106FCCDC030E0101F8
:100D6C000D6F010E0E6F270E0F6F000E106FC2DC91
:100D7C00040E01010D6F010E0E6F150E0F6F000E9C
:080D8C00106FB8DCFFD7FFD7A0
:1010720010EE15F0460E006E010E016EE10EF66ED8
:0E1082000D0EF76E000EF86E62EC03F0120019
:100D9400204469726563746F7279203A433A5C5FE8
:100DA4004D696B726F435C5F4D657350726F6A651A
:100DB40074735F4D696B726F435C5F4C6973745FEE
:100DC4004932435F646576696365735F6F6E5F7410
:0D0DD40068655F4932435F4275730D0A0088
:100DE1007061756C666A756A6FE0667265652E661C
:020DF10072008E
:100DF300466F6320696E7465726E652031364D48A7
:020E03007A0073
:040E050000000000E9
:010E090000E8
:0F0E0A005049432031384634364B3232202000D5
:0E0E190049324331204C4344203478323000BB
:100E2700204C4344203478323020493243202C2050
:100E37006D6F64756C652020454570726F6D20324B
:100E4700344C433332206176656320525443204447
:100E5700533133303720737572206C6520427573B8
:020E6700200069
:100E69002050726F6A6574203A5F31384634364BC8
:100E790032325F4C6973745F493243315F6F725F1D
:100E8900493243325F646576696365735F6F6E5F8C
:100E99007468655F6275732E6D63707069200D0AE1
:010EA9000048
:100EAA00204176656320522070756C6C2075702025
:100EBA00646520322C374B20737572206C65732061
:100ECA006C69676E65732053434C206574205344E4
:100EDA00412064752062757320493278200D0A001A
:100EEA0020536F75726365203A205F313846343675
:100EFA004B32325F4C6973745F493243785F646581
:100F0A0076696365735F6F6E5F7468655F62757338
:0C0F1A005F3138303430392E630D0A008E
:100F26000D0A4C69737420577269746520416472A6
:100F36006573732049324378204465766963657327
:100F4600202866726F6D2040333220746F20323550
:070F56003429203A0D0A00C6
:100F5D00204C656374757265206164726573736589
:100F6D00732064657669636520737572206C6520E6
:100F7D006275732049324331206F752049324332F7
:050F8D0020200D0A0008
:100F920020496E6974204932433120205243333D47
:100FA20053434C31205243343D534441312031307C
:080FB200304B687A200D0A00A3
:100FBA0020446576696365202320202066696E6473
:0E0FCA002061742040202020202020202000C4
:100FD800204D6F64652042417661726420736920F8
:0A0FE800524135203D30200D0A0073
:100FF200204D696B726F432070726F20372E313033
:04100200200A0D00B3
:10100600204D6F64652042617661726420524135DD
:03101600203D007A
:101019002050726573656E746174696F6E3A200D44
:021029000A00BB
:10102B003031323334353637383941424344454613
:10103B00204465766963652023202020403D2000F5
:0B104B0020493243202331200D0A0011
:0B105600206E6F7420666F756E6400E2
:0A10610044657669636520402000B5
:07106B0020736F697420007F
:020000040030CA
:0D000100281F3CFFBF81FF0FC00FE00F4024
:0200000400F00A
:10000000FFFFFFFFFFFFFFFFFFFFFFFFFFFFFFFF00
:10001000FFFFFFFFFFFFFFFFFFFFFFFFFFFFFFFFF0
:10002000FFFFFFFFFFFFFFFFFFFFFFFFFFFFFFFFE0
:10003000FFFFFFFFFFFFFFFFFFFFFFFFFFFFFFFFD0
:100360007061756C666A756A6F200A0D00FFFFFF89
:10037000FFFFFFFFFFFFFFFFFFFFFFFFFFFFFFFF8D
:10038000FFFFFFFFFFFFFFFFFFFFFFFFFFFFFFFF7D
:10039000FFFFFFFFFFFFFFFFFFFFFFFFFFFFFFFF6D
:1003A000FFFFFFFFFFFFFFFFFFFFFFFFFFFFFFFF5D
:1003B000FFFFFFFFFFFFFFFFFFFFFFFFFFFFFFFF4D
:1003C000FFFFFFFFFFFFFFFFFFFFFFFFFFFFFFFF3D
:1003D000FFFFFFFFFFFFFFFFFFFFFFFFFFFFFFFF2D
:1003E000FFFFFFFFFFFFFFFFFFFFFFFFFFFFFFFF1D
:1003F000FFFFFFFFFFFFFFFFFFFFFFFFFFFFFFFF0D
:00000001FF
